:020000040000FA
:100000000428FF3FFF3FFF3F07300313831299008F
:1000100083169F010F30850005308312CB00D52356
:100020000B24AA30D000F1228730D000F122013019
:10003000D000F122C12376233430FB00FF30FA00D8
:10004000FB0B23282628FA0B23282028CF30FA0080
:10005000FA0B282800005030B0006130B100BD30EC
:10006000B200B530B3000230A200063022020318FD
:100070004D2802302202F000F101031CF103700848
:10008000343FC700F8302207CB005C2483124708B6
:10009000840070088000A20A35283A08F300390865
:1000A000F2003808F100F0013408F800F901FA0113
:1000B000FB017008F80771080318710FF90772083F
:1000C0000318720FFA0773080318730FFB077808F9
:1000D000B8007908B9007A08BA007B08BB007A0832
:1000E000F3007908F2007808F100F0013508F80013
:1000F000F901FA01FB017008F80771080318710F84
:10010000F90772080318720FFA0773080318730FC0
:10011000FB077808B8007908B9007A08BA007B08AC
:10012000BB007A08F3007908F2007808F100F001CA
:100130003608F800F901FA01FB017008F8077108A8
:100140000318710FF90772080318720FFA07730882
:100150000318730FFB077808B8007908B9007A080C
:10016000BA007B08BB007A08F3007908F20078082F
:10017000F100F0013708F400F501F601F70170080D
:10018000F40771080318710FF50772080318720F4E
:10019000F60773080318730FF7077408B80075089B
:1001A000B9007608BA007708BB0077083302031D50
:1001B000E32876083202031DE32875083102031D87
:1001C000E32874083002031CFB283008AC00310817
:1001D000AD003208AE003308AF003808AC02390871
:1001E000031C390FAD023A08031C3A0FAE023B085C
:1001F000031C3B0FAF0233083B02031D09293208E1
:100200003A02031D092931083902031D0929300862
:100210003802031C21293808AC003908AD003A081F
:10022000AE003B08AF003008AC023108031C310FB0
:10023000AD023208031C320FAE023308031C330F29
:10024000AF0229082A06031D31290F300505F000E9
:100250007008AB00F0097008AB000F307005A90002
:1002600021292908AA003430FB00FF30FA00FB0BDB
:100270003A293D29FA0B3A293729CF30FA00FA0BEF
:100280003F2900007529BC01B6290630BC00B629FB
:100290000C30BC00B6291230BC00B6291830BC00A6
:1002A000B6291E30BC00B6292430BC00B6292A303D
:1002B000BC00B6293030BC00B6293630BC00B629A7
:1002C0003C30BC00B6294230BC00B6294830BC00E6
:1002D000B6294E30BC00B6295430BC00B6295A307D
:1002E000BC00B629F830BC00B6292908003A031929
:1002F00043292908013A031945292908023A031913
:1003000048292908033A03194B292908043A0319F3
:100310004E292908053A031951292908063A0319D3
:1003200054292908073A031957292908083A0319B3
:100330005A292908093A03195D2929080A3A031993
:10034000602929080B3A0319632929080C3A031973
:10035000662929080D3A0319692929080E3A031953
:100360006C2929080F3A03196F297229A201063056
:1003700022020318C92922083D3FC7003C08220772
:10038000CB005C2483124708840070088000A20A16
:10039000B7293430FB00FF30FA00FB0BD029D329FA
:1003A000FA0BD029CD29CF30FA00FA0BD52900005D
:1003B0004508CA004408C9004308C800C701023004
:1003C0003C07CB005C247008F400F501F601F7014E
:1003D00083124708F40748080318480FF50749082F
:1003E0000318490FF6074A0803184A0FF70774085D
:1003F000C3007508C4007608C5007708C6007608F3
:10040000CA007508C9007408C800C70103303C075A
:10041000CB005C247008F400F501F601F7018312AB
:100420004708F40748080318480FF5074908031858
:10043000490FF6074A0803184A0FF7077408C30064
:100440007508C4007608C5007708C6007608CA009B
:100450007508C9007408C800C70104303C07CB0008
:100460005C247008F400F501F601F70183124708D7
:10047000F40748080318480FF50749080318490FFF
:10048000F6074A0803184A0FF7077408C3007508EF
:10049000C4007608C5007708C6007608CA0075084B
:1004A000C9007408C800C70105303C07CB005C24B4
:1004B00070088312C300C401C501C6014708C30701
:1004C00048080318480FC40749080318490FC5070F
:1004D0004A0803184A0FC6073B083302031D7A2A4D
:1004E0003A083202031D7A2A39083102031D7A2A9A
:1004F00038083002031C8A2A2C08C3022D08031C6A
:100500002D0FC4022E08031C2E0FC5022F08031C3A
:100510002F0FC60233083B02031D982A32083A0205
:10052000031D982A31083902031D982A3008380221
:10053000031CA82A2C08C3072D0803182D0FC40775
:100540002E0803182E0FC5072F0803182F0FC607F4
:100550004308C2004408C1004508C0004608BF0067
:1005600028240730A20022080C3C031CCD2A0B24AF
:10057000AA30D000F1222208D000F1220730220256
:10058000F000F101031CF10370083D3F84000008F6
:10059000D000F122C123A20AB32A1A245024A201B6
:1005A000063022020318EF2AF0302207CD0022087D
:1005B0003D3F84000008CE00A7233430FB00FF300D
:1005C000FA00FB0BE42AE72AFA0BE42AE12ACF30EF
:1005D000FA00FA0BE92A00008312A20AD02A212984
:1005E000F02A083003138312D100D20120088400BE
:1005F000831351080319162B66246624FB238012EB
:10060000662450080319042BFB23D00D031C0B2B6D
:10061000841700160D2B8417001200006624801624
:100620008413801E112B8417D103F92AD20166246A
:10063000FB230000801266240016662466245208FC
:100640000319222B80168413801E242BD2016624CA
:100650008413001A521466246624662466246624D1
:10066000662466246624FB23841780120012520835
:10067000F0000800083003138312CE00CF012008D9
:10068000840083134E08003C03185C2B6624000092
:10069000001666244F0803194D2B80168413801E04
:1006A0004F2B001A0314001E0310CF0D6624FB23EA
:1006B00084178012CE03422B001666244D080319BE
:1006C000622BFB234D080319662B001200006624E1
:1006D00080168413801E6A2B84176624FB238012E5
:1006E0006624FB2300124F08F000080007300313B4
:1006F0008312CD004324A2012208053C031C962B43
:100700002208233FCB000130CD003A234B08840060
:1007100070088000F8302207CD002208233F8400B3
:100720000008CE00A7238312A20A7C2B2208013FD7
:10073000F000F1010318F10A7008233FCB00CD014E
:100740003A234B08840070088000C1230800000091
:10075000031383169C1CAE2B0000A82B83124D089C
:1007600083169B0083124E0883169A009C131C1557
:100770008B1355309D00AA309D009C148B171C11C3
:10078000080003138312200884008313FB23001244
:10079000662480168413801ECB2B8417662466245F
:1007A00066246624001666240800031383124B088F
:1007B00084000008CC004C12CC124C088000841736
:1007C0000408A000001680168413801EE52B080084
:1007D000003003138312A2000030A900FF30AA00EA
:1007E0000030AB000030AC000030AD000030AE0097
:1007F0000030AF000800040803138312D40020085F
:10080000840084130008D3005312D31253088000CD
:100810005408840008000313831220088400831303
:100820000016662480166624FB2300126624FB2330
:1008300080120800893003138312CD004324CD01B8
:100840003A237008A100EF307005A100362408009B
:10085000893003138312CD004324CD013A2370085D
:10086000A10010307004A10036240800C1230B241D
:10087000AA30D000F1228930D000F1222108D00026
:10088000F122C12308000B24AA30D000F1224D0828
:10089000D000F122C1230B24AB30D000F12208009C
:1008A0000B24AA30D000F1228730D000F122403052
:1008B000D000F122C1230800031383124B088316D2
:1008C0009B009C131C141A08F00008000000000094
:1008D0000800FF3FFF3FFF3FFF3FFF3FFF3FFF3F5E
:1008E000FF3FFF3FFF3FFF3FFF3FFF3FFF3FFF3F18
:1008F000FF3FFF3FFF3FFF3FFF3FFF3FFF3FFF3F08
:10090000FF3FFF3FFF3FFF3FFF3FFF3FFF3FFF3FF7
:10091000FF3FFF3FFF3FFF3FFF3FFF3FFF3FFF3FE7
:104200004E004200AD00DB003A00510015004200B4
:10421000A900D3003700DE003000C200A900210051
:104220007B00B6006B00C200A80044002C00AE006A
:104230006B00C200AF006A0045008100E700420049
:10424000AA0029003800120014004200AD0001004D
:104250005B00EF006B004200A70053005F004F00BF
:104260002F00C200A900EA002600DB00E300C20024
:10427000B500BD0061003E00E300C200B9007C0053
:1042800000008700E300C200BD003A009F00D1009B
:1042900028004200A800F000BF00DD002800420016
:1042A000AC008E00B000FF004400C200A700F10087
:1042B0009D0020004400C200A90049009D00F100BB
:1042C0004E004200AD00DB003A005100FF00FF004D
:1042D000FF00FF00FF00FF00FF00FF00FF00FF00E6
:1042E000FF00FF00FF00FF00FF00FF00FF00FF00D6
:1042F000FF00FF00FF00FF00FF00FF00FF00FF00C6
:10430000FF00FF00FF00FF00FF00FF00FF00FF00B5
:10431000FF00FF00FF00FF00FF00FF00FF00FF00A5
:10432000FF00FF00FF00FF00FF00FF00FF00FF0095
:10433000FF00FF00FF00FF00FF00FF00FF00FF0085
:10434000FF00FF00FF00FF00FF00FF00FF00FF0075
:10435000FF00FF00FF00FF00FF00FF00FF00FF0065
:10436000FF00FF00FF00FF00FF00FF00FF00FF0055
:10437000FF00FF00FF00FF00FF00FF00FF00FF0045
:10438000FF00FF00FF00FF00FF00FF00FF00FF0035
:10439000FF00FF00FF00FF00FF00FF00FF00FF0025
:1043A000FF00FF00FF00FF00FF00FF00FF00FF0015
:1043B000FF00FF00FF00FF00FF00FF00FF00FF0005
:1043C000FF00FF00FF00FF00FF00FF00FF00FF00F5
:1043D000FF00FF00FF00FF00FF00FF00FF00FF00E5
:1043E0006800C200A9007C0082007400FF00FF008A
:1043F000E100C200B500F0004500D300FF00FF005F
:02400E00C43FAD
:08400000FF3FFF3FFF3FFF3FC0
:00000001FF
